:0C000000830100308A0004288301992B42
:100718008312BE000430BF005330C000C00B922BC0
:10072800BF0B902BBE0B8E2B0800FF3083128E0060
:1007380002308F000C30900002309100FF309200A0
:1007480093019400893095009600970081309800B5
:100758009901FF309A0011309B0031309C005130D4
:100768009D008E309E009F01FF30A0001030A10038
:10077800A200A300FF30A400A501FC30A60012309F
:10078800A7001130A8001230A900FC30AA00AB0164
:10079800FF30AC008930AD00AE00AF007630B0005D
:1007A800B101FC30B2001230B3001130B400123085
:1007B800B500FC30B600B701B801B901BA01BB01F8
:1007C800BC01BD018316860183128C018D010C08C2
:1007D8000E3E840000088600013083128C238C0AA8
:1007E80003198D0A00300D02303003190C02031C66
:0807F800EB2B30308C23E82BC1
:00000001FF
